:10000000FF23831690001F30850087010030831284
:10001000A500DF115F110030AD000030AE00662199
:10002000AC0000308A002C0EB400B40C340C033940
:100030001A3E82001E284B284B284C2800308A008C
:100040002C0CB400B40C340C0739273E82002F2846
:100050004A284A284A284A284A284A284A28003052
:100060008A0007302C05353E82003D284028432871
:100070004628492849284928492827088F214928FE
:1000800025088F21492824088F2149286621A500A9
:1000900049284A28BA28BA2800308A002C0CB40013
:1000A000B40C340C0739553E8200BA28BA28BA2855
:1000B000BA28BA285D286B28842807302C05F93E19
:1000C000031D6A280030B100DF19B1145F19311423
:1000D00031088F21BA2800308A002C0C0339713E78
:1000E0008200752875287C288028DF11AC18DF1560
:1000F0005F112C185F1583285F112C185F1583285A
:10010000DF112C18DF15BA2800308A0007302C05C3
:100110008A3E8200922896289A289F28A228AF28F3
:10012000B228B7288316FC309007BA28831604300B
:100130009007BA288316100883128F21BA2800303E
:100140008F21BA280030B20032302E020318AC28BA
:100150002E082E21B200AE0A32088F21BA280030B4
:10016000AE00BA282D088F210030AD00BA282D0A24
:10017000031DAD0A83120F28640033300505333A9E
:10018000A400013024050319E028C628C728000070
:10019000023024050319D328CD28CE280130A7002A
:1001A0000230A600DF2810302405031DDB28A7013C
:1001B0000130A600DF280730A7008030A6001A29EA
:1001C00020302405031DFF28023024050319F028E0
:1001D000E928EA2800000230A7000430A600FE2823
:1001E00010302405031DF928FF30A700FF30A600BA
:1001F000FE280630A7004030A60000001A29023071
:10020000240503190B290429052900000330A70040
:100210000830A600192910302405031D14290430C4
:10022000A7001030A60019290530A7002030A6002D
:100230000000000025082605031D5F15DF1923298E
:100240002929222929295F1927290000292905118F
:10025000DF111B30FF3E031D2A29003484000130CA
:100260008A000408343E820001340034163400341D
:1002700000340034003400340034003400340034DE
:1002800000340034003400340034003400340034CE
:100290000034003400340034093443346F346D3496
:1002A0007034613473347334383444340F34473425
:1002B000723461346D346C34693463346834263498
:1002C000423465346E3473346F346E34DF145F142B
:1002D000851D6C29BC206829DF100515BC20BC20B9
:1002E000BC200030A100742975297629000008304F
:1002F000B500BC20A10CA1138519A117BC20BC20FE
:1003000081298229B50B7929BC20BC2087290000CE
:100310002908A8002108A900051521080800A30044
:100320002B08AA002308AB005F1C9C295F100A3031
:10033000B600BC20B60B99290511BC20BC20BC20FE
:100340000230FF3E031DA1290830B6002318051511
:10035000231C0511A30CA313BC20BC20BC20B02976
:10036000B60BA6290515BC20BC20BC200230FF3EE0
:08037000031DB729BB2900346D
:02400E009431EB
:00000001FF
